:020000040000FA
:060000000219FD0200B32D
:03002B0002008D43
:03005B0002028C12
:030073000200A0E8
:100080000406080C10182030406080A0C0C0D0C00A
:10009000E0C2CF0541E52360021523D0E0D0D03285
:1000A000C2AF53E67F7592FA7593FFC22053917FDA
:1000B000D2AF32C2AF53E6EFC0D0C0E0C0F0D2D36F
:1000C000D2AF5388EFA88AA98C758A00758C00433B
:1000D000881030331FE8C4540FFAE9C454F04AFAC8
:1000E000C3132AFAC3E833F8E933F9E82AFAE93402
:1000F00003FB213D30320FC3E833E933FAE82AFA33
:10010000E93400FB213D303115E875F056A4AAF022
:10011000E975F056A42AFAC5F03400FB213DE875D4
:10012000F02BA4AAF0E975F02BA42AFAC5F034004C
:10013000C313FBEA13FAC3EB13FBEA13FAC3EB9402
:10014000095006C3EB9403501A0522E522700215EC
:1001500022C3E522940A5002417F7552007A007B47
:1001600000414DE522600215223035067C007D04F9
:10017000217DAC31AD32303A04AC33AD34C3EA9CAE
:10018000FAEB9DFB9208AE5EAF5F303A425007201B
:100190003409D234219B303402C234303404AE608E
:1001A000AF61203902B234C3EA33FAEB33FBA20861
:1001B000500AEAF42401FAEBF43400FBC3EA942871
:1001C000FAEB9400FB501478007A007B0021DBA24C
:1001D00008500878007A007B004131E5255403601F
:1001E00019202A16E55BF9EB7007C3E99A4002E98A
:1001F000FAE53CC42AFAEB3400FBEA8EF0A4F9AA33
:10020000F0EB8EF0A42AFAC5F03400FBC3EB13FD2B
:10021000EA13F80FEF146004C3E833F8C3E933EAD4
:1002200033FAEB33FBDFEDEB30E20678FF7AFF7B4E
:10023000038852D230C3E559FC955A4002AC5AC3E8
:10024000EC95525008EC75F004A4FAABF0EAF4F81F
:10025000EBF45403F9C3E8940FFAE99400FB50045B
:100260007A007B00885489558A568B5775230AD0AB
:10027000F0D0E0D0D053F7DF43F74043E6103275BB
:10028000230AD0F0D0E0D0D043E61032C2AF53A85A
:10029000FEC0D0C0E0D2D3A8F9E55830E10AE5FAB3
:1002A00020E14220E03F41B0E5FA30E13820E0357E
:1002B000C3E55513F8E55413F5FB88FCC3E5571364
:1002C000F8E55613F5E988EA85555853F7BFC3E5B5
:1002D000529401400575530041E5E5532401F5535F
:1002E00050037553FF53F7DFD0E0D0D043A801D2BD
:1002F000AF327901801479038010790A800C791E5D
:1003000080087964800479C880007817E4D5E0FD1E
:10031000D8FAD9F6227A147B7880127A107B8C80F6
:100320000C7A0D7BB480067A0B7BC88000E562D521
:10033000E001227902E4C291D5E0FDD290D5E0FD42
:10034000C290D5E0FDD291D5E0FDE920E002D28651
:1003500030E002D292E562D5E0FDE920E002C286FB
:1003600030E002C2927496D5E0FDD9C9EAF8D5E032
:10037000FDD8FBDBB8C2912278FF20282879A1E7BD
:100380006023E548601F74FF8548F084853FF030A6
:10039000290375F005A4F8C5F0600278FFC3E8955D
:1003A0005B5002A85B885A22C3E54794E4E5489471
:1003B00000E55A50031461B9046002F55A2275E849
:1003C0009022055CC3E55C9408405330EDF4A8BD71
:1003D000A9BE755C00E9FA79A0E76041EA7006E51C
:1003E0005D6018800CC3E8955D600EE55D500560AA
:1003F0000A1480070460FA8002E55DF55DC3956725
:10040000401B7559C0C394044013755980C39404AC
:10041000400B755940C39404400375590022E559B7
:100420002410500274FFF55922743279A687F0A483
:10043000C5F0A2F733F8C3E895594002A859885B84
:10044000227547007548F022C2AF75C800A8CCA934
:10045000CDAA4130CF010A75C804D2AFAB42AC433C
:1004600088428943C3E89BF8E99C202808F9302C8E
:1004700002A15781B1AD448A44F9EA9DFA6004783B
:10048000FF79FFAE45AF468B458C46A842A943C3D2
:10049000E89EF8E99FF9C3E54813FBE54713FAE83E
:1004A0002AF547E93BF54850067547FF7548FF8137
:1004B000FEAA47AB48AC47AD487E047F02C3EB942D
:1004C00004400D1E1FC3EB940840052029021E1F87
:1004D000C3ED13FDEC13FCDEF7C3EA9CFAEB9DFBC6
:1004E000EF6009C3E913F9E813F8DFF7EA28FAEB3C
:1004F00039FB8A478B4850067BFF8B478B48C3EB01
:1005000094025002D22C3028047F03A1297892E66D
:10051000FFC3E53D948240110FC3E53D94A0400127
:100520000FC3EF940640027F057E02E548C4540FD6
:10053000F9E548C454F0F8E547C4540F28F8C3E877
:100540009EFAE99400FB4009C3EA9401EB94005041
:10055000047A01E4FBA1A3AA47AB48EBC4FEEAC4BA
:10056000540F4EFCC3EA9CFAEB9400FBC3E813C3A0
:1005700013F8EA28FAEB3400FB8A478B48C3EB9464
:10058000024002C22C7802EBC4FE7B00EAC4540F86
:100590004EFAC3EA98FA4005C3940150027A0178F2
:1005A00092E6FF302002A1A3854E92854F93D22080
:1005B00043E680C3E49AF8E49BF9302C02C12EE8AC
:1005C000FAE9FBD3E913FDE813FC884E894FC3EF2A
:1005D00094036037EF20E00CE82CF8E93DF9ECFAE1
:1005E000EDFB8013E828F8E939F9C3E82401F8E9BC
:1005F0003400F97AFF7BFFC3EF9403400E8A508BDF
:1006000051884A894B8C4C8D4DC162885089518AE2
:100610004A8B4B8C4C8D4D3028127550F07551FF24
:10062000754CF0754DFF754EF0754FFFC162E8FADD
:10063000D3E813FC884EC3EF94036020EF20E0075B
:10064000E82CF8ECFAC14EE8282401F87AFFC3EF51
:10065000940340088A50884A8C4CC16288508A4A68
:100660008C4C302002C162753A02D22043E680E50C
:100670002554036034A847A948C3E913F9E813F8DF
:10068000C3E913F9E813F8302804E92440F9C2AFAC
:1006900053E67F759100C3E498F594E499F5957558
:1006A0009104D22043E680D2AF22D2217549007551
:1006B0002000302B03752040800ED2217549007533
:1006C0002040302B0375200078017901202C20E593
:1006D0002554036002C2217914E548C31370010454
:1006E000F8C3941440027814302804781B791B2036
:1006F0002010E549600C302803D53A04D223E1727A
:10070000D16A0549E59B5440B52002E15C302809D7
:1007100008C3E899400118C1EF20210A08C3E899ED
:100720004002C1C8C1EFC221C2AF53E67F7591003C
:10073000302C127594007595F8759104D22043E61B
:1007400080D2AFC1C8E5487EFFC3334005C3334004
:1007500001FEC3E49E759400F595E139C3E5399433
:10076000015002C1C8302102C1C8D802E170C1EFF6
:10077000C223C2AF53E67F75910085509485519591
:10078000759104854A92854B93D22043E680D2AF7F
:10079000E525540360072029020539801030230D18
:1007A000202B0A20210715811581020EB622780020
:1007B0003021027801E53D75F007A4F9E5F028F550
:1007C000F0E9A2F013A2F113A2F213F53DC394785D
:1007D0005003753D78C3E53D953E400ED222C2865A
:1007E000C290C29275D4FF75D50F302002E1EA8520
:1007F0004C92854D93D22043E68022203813C2AF1D
:10080000C291D28775D4FF75D503D2AF759F4201CF
:10081000F3C2AFC291D29375D43F75D50FD2AF75E5
:100820009F4201F3203814C2AFC29275D4FF75D530
:100830000CD287D2AF759F520208F3C2AFC2867541
:10084000D4FF75D50CD293D2AF759F320208F32036
:100850003813C2AFC287D29375D4FF75D50CD2AF0F
:10086000759F3201F3C2AFC293D28775D4FF75D59D
:100870000CD2AF759F52807B203814C2AFC29075E6
:10088000D43F75D50FD293D2AF759F420208F3C201
:10089000AFC29075D4FF75D503D287D2AF759F4292
:1008A0000208F3203813C2AFC293D29175D43F75BA
:1008B000D50FD2AF759F52803AC2AFC287D2917521
:1008C000D4FF75D503D2AF759F328027203813C26D
:1008D000AFC28675D4FF75D503D291D2AF759F3262
:1008E0008011C2AFC29275D43F75D50FD291D2AFED
:1008F000759F52C22222C286C290C292C287C29102
:10090000C29375D4FF75D50F22788076FF0876FFE5
:100910000876FF0876FF0876FF0876FF0876090854
:1009200076FF087601788C76010876FF0876FF0856
:1009300076FF0876FF0876FF0876030876FF0876CC
:10094000FF0876FF0876250876D0087628087650C6
:100950000876040876FF0876020876FF08767A089B
:1009600076FF0876070876010876FF0876FF087696
:100970000008760022FA75F00CA4ABF0EAC333F855
:10098000740133F9E8C333F8E933F9E8C32BF8E924
:100990003400F9227888E6C39403D23A5002C23A6E
:1009A000C238E630E102D238A23892397886E614AD
:1009B0009000809378A6F67886E6F53FC3940250BF
:1009C00003753F02789CE6753EFFB40203753EA0B6
:1009D000B40303753E8278A0E6F860067428240903
:1009E000D8FCF5677896E6317588318932789EE6CD
:1009F0003175883389347897E631758835893611B1
:100A0000F6223035117A007B007CFF7D007E00519C
:100A1000698B5F8A5E22303A227896E6FA7B00780C
:100A20009EE6FC7D00C3EA33FAEB33FBC3EC33FCF8
:100A3000ED33FD7E0A51698B618A607896303A0207
:100A4000789EE6FA7B007897E6FC7D007E00303ADF
:100A500010C3EA33FAEB33FBC3EC33FCED33FD7E1A
:100A60000A51698B5F8A5E2222C3EC9EFCED9400E2
:100A7000FDC3EC9AFCED9BFDC3EC9423ED94005078
:100A8000047C237D00C3EC94FFED940140047CFFC3
:100A90007D017BFF0B7A000AEA7009C3EC33FCEDA1
:100AA00033FD4194EC8AF0A4AEF0ED8AF0A42E94CC
:100AB0007C40E4EAF460DD22D23551021202FE12DB
:100AC00002FE7A007B007C101202F6E5522AFA74CC
:100AD000003BFBDCF37C04C3EB13FBEA13FADCF70B
:100AE000FFEB60027FFFC23551022278A5E6F95480
:100AF000037000E9540C7000E954307000E954C0F0
:100B00007000227565007566007597DE7597AD7586
:100B100081C043FF8075EF0675A90011F675803F0F
:100B200075F1C375A4C075803F75D4FF75900075CD
:100B3000F20F75A50F75900075D50F75A60175E3B9
:100B40004075E20211F6E4F8F6D8FD3109D1E878F3
:100B5000988662753001C2AF1203061203151202A5
:100B6000FE12031B1202FE1203211202FE51EBC2FF
:100B7000AF75650075660078FA79FA308007D9FBA1
:100B8000D8F7021C00319451027898866211F675EC
:100B9000E400758811758E0475890975C80475910E
:100BA0000475D84075D90875F781759E037596024E
:100BB00075DA4275DB4275A82175E69075F31075FC
:100BC0009B80759D0075D10C75BC5975BB1075E87F
:100BD0008075B2011202F2D2AF753C00C23012032E
:100BE00006C231752200120302C3E522940A402492
:100BF000D231C232752200120302C3E522940A40A8
:100C000013D232C233752200120302C3E522940AC2
:100C10004002D2331202F6203003020B6FC2AF1231
:100C20000315120315120315D2AF120306303A0250
:100C300081D11202F6788CE6C39401500281D1E58D
:100C400030C39401500281D17565A57566F17F02AC
:100C5000D2355102120302C2AFC2355102C3E5526E
:100C6000947FD2AF406B1202F2C2AF120327D2AF11
:100C7000DFDE51B8C3EF7897F6120306F1C87F0A9A
:100C8000D2355102120302C2AFC2355102C3E5523E
:100C9000947FD2AF50E81202F2C2AF1203151202D3
:100CA000FA120315D2AFDFD851B8EF24037896F6C5
:100CB000F87997E7C394234003985006E8242378F3
:100CC00097F6120306F122120FF712030251026186
:100CD0006F7565007566001203027801303A02787C
:100CE00005C3E552984002812DC2AF1203271203BB
:100CF00027120327D2AF120306753000E4F537F54B
:100D0000380537E537F4703E0538789AE6781914D7
:100D10006012783214600D787D14600878FA1460DF
:100D200003753800C3E53898401C11F61202F2151D
:100D30003875370078998662C2AF120327D2AF7830
:100D40009886621203021202FAE5237002616F783C
:100D500001C3E5529840AA120302E5237003020B77
:100D60006FC2AF11F6E4D2AFE4F55CF524F525F5DA
:100D70003D755C081202F21203BE30EDFDA8BDA95C
:100D8000BEE97001F8885D1203C2755C08C2AF75D8
:100D900059FF120429855B59855B5AD2AF303A0757
:100DA000C238303402D238D22875390011A311CCA0
:100DB0001204411204481204411204481204411260
:100DC00006BA1207AE1207FB1204481206AA202C1C
:100DD00003120378302C031203A81207AE11241259
:100DE00004481206BA1207AE114F1204481206AA9E
:100DF0001207AE11781204481206BA1207AE11A3F8
:100E00001204481203BE1206AA1207AE11CC120336
:100E1000C2120448302827855B5979187A0CC3E53B
:100E20003999400EC228D2298A3B855B59855B5A85
:100E3000800CC3E55294014003020DBFC1BE3029AE
:100E40001C202B19E53B147006C229D22AA1BFF53C
:100E50003BC3E55294014003020DBF8061753C0025
:100E600078FA79A4E760027803C3E55398504FE518
:100E700023604B303A17203805203407800F303478
:100E800002800A202B07D22B855B59A1ED78F03028
:100E90002B05855B597820C3E548985003020DBFA8
:100EA000302B1BC22BC238303402D238D229753BCA
:100EB00012855B59A1BF053CE5526002C1C1753C7A
:100EC00000C2AF11F6752400752500D2AF120302DF
:100ED00011F678A4E66006D287D291D293C3E53C9E
:100EE00094044002616F81FC901A0D7820F15BE55B
:100EF00020B4550AA3F15BE520B4AA0280063109AB
:100F0000F122801D901A0378807B0AF15BA308DB35
:100F1000FA901A0F788C7B1AF15BA308DBFA901A0F
:100F20002922C2AFF19EF17B901A007410F160A3E8
:100F30007403F160A37421F160901A0378807B0A36
:100F4000F15FA308DBFA901A0F788C7B1AF15FA38C
:100F500008DBFAF1B1F18F901A2922E493F622E628
:100F6000438F01538FFDFFC3E583941C400122EFA3
:100F70008565B78566B7F0538FFE22438F02438F96
:100F8000018565B78566B7901A0DF0538FFC2290E6
:100F90001A0D7455F160901A0E74AAF160227A301D
:100FA00079D07820901A40F15BE520F709A3DAF7B1
:100FB000227A3079D0901A40E7F16009A3DAF92259
:100FC0007C05120306DCFB22C2AF12031512031BC1
:100FD0001203211203271202FA12031512031B1225
:100FE00003211203271202FA12031512031B120324
:100FF00021120327D2AF22C2AF12032712032112FC
:10100000031B1203151202FA120327120321120303
:101010001B1203151202FA12032712032112031BDB
:06102000120315D2AF22FD
:1019FD00020B03100321FFFFFFFFFFFF09FF01FF94
:101A0D0055AA01FFFFFFFFFF03FFFFFF25D0285061
:0D1A1D0004FF02FF7AFF0701FFFF0000FF3A
:101A400023435F4C5F31352320202020202020209D
:101A500023424C48454C492445464D3842313023B9
:101A60002020202020202020202020202020202076
:101C0000C2AFC2D37597DE7597AD7581C075A90057
:101C100043FF80752438752503B1DB7529A5752A26
:101C2000F143F10153A4FED28075D4FF75E3407DEA
:101C3000FA780379E67C10752200752300901DE880
:101C40007B06752498752501308002814820800824
:101C5000D8FBD9F9DCF781BA308008D8FBD9F9DC98
:101C6000F781BAB19BE493A3C39A6004DDC381BA40
:101C7000DBDBB18D600281317B08E493FAA3B16EA6
:101C8000DBF87A30B16E752200752300B18DEAFC65
:101C9000EBFDC3ED94FE400EB18D8A278B28ED300D
:101CA000E0048A828B83B18D7AC270D8C3ED94FE32
:101CB000601950CEBD0029EC600F7520007521FF22
:101CC000752900752A000200008100A827A92808AC
:101CD00009D804D90281DDB191EAF281D10D81A642
:101CE000C3ED94035051EDA2E092007AC5C3E582A2
:101CF0009400E583941C508C200010438F02438F86
:101D0000018529B7852AB7F0300027A827A9280818
:101D100009438F01538FFDD804D902A132C3E58353
:101D2000941C4003A3A117E28529B7852AB7F0A325
:101D3000A117538FFC81827AC1BD030CE493A3FAEF
:101D4000B152DCF8B14A81828184AA22AB23B16E00
:101D5000EBFAEA6222752608C3E52313F523E52290
:101D600013F52250066323A0632201D526EAB1DBD6
:101D7000B1DB75260AEAF4200102D280300102C2EA
:101D800080B1DBC3134002C201D526EB22B191EA38
:101D9000FB208002A191308002A196752608AE2416
:101DA000AF25C3EF13FFEE13FEB1DFB1DBC3EA13C0
:101DB0003080024480FA30E703632201C3E5231335
:101DC000F523E52213F52250066323A0632201D5F3
:101DD00026D9E52265236523F52222AE24AF250E00
:101DE0000FDEFEDFFCD20122424C48656C693437BD
:061DF0003163E8B10601B9
:00000001FF
